:020000040000FA
:020000001628C0
:080008009A2D82073F340634F3
:100010005B344F3466346D347D3407347F346F3451
:1000200000340234043408341034203403138312AF
:100030008501860187019F018316031788018901C5
:10004000031375308F007030850001308600870102
:1000500008308900C33081000C10831200308B00FF
:10006000013090008601861700003230051B3C30BD
:10007000A100A3000310A30CA30C0B160B178B17E6
:100080008030A20086018614221C871422180714CF
:100090007F258701860106170000051F422886017B
:1000A000A2012108A3002030A600A7000730A80065
:1000B0002630A900CA011230AA00AB01AC01013000
:1000C000A40091265008A500B501B801B701BB01F5
:1000D000B901BD01BE01C901A03084003C30C1009E
:1000E0008001840AC10B7028891DBE173B1706309A
:1000F0008100FA30A0008B1638189928B401B2019B
:100100002408BE1B25089823CA188E282A08B00088
:100110002B08B100BE1BBE1DE92399284A1A952859
:100120002608B0002708B10099282808B00029083F
:10013000B100C030BB05023086000130CA18A528C6
:1001400002304A18A5283208A7284A1D0301870053
:100150007F255121003087000430860031080F3997
:100160000520CA1EB6284A1DBA28B928BE1FB928BC
:100170003E1A803887007F255121003087000830E3
:100180008600310E0F390520BE1FC9284A1AC9281A
:100190003E1A803887007F255121003087001030BB
:1001A000860030080F39052087007F255121003057
:1001B000870020308600300E0F39031DE828CA184A
:1001C000E8284A18E8283E1BE828BE1BBE1D0A3056
:1001D000052087007F2551210030870040308600B0
:1001E000330887007F25512100308700803086004A
:1001F000340887007F2551210030870086013B08A5
:10020000C039031916293B1B07297E211629BB1B60
:1002100016293B081F39153C031D16292008031D0C
:100220001629063081004B30A0008B1637189B240E
:100230003E1F2A29BF0A0030BF1BAA30B000B10000
:100240003F08031D2A29BE0307303E05031D2A2946
:100250003E13B8018B1A5029490803195029491F28
:1002600036295F2587255F25BB014F29C91E3B29FC
:100270005125BB014F29491E40294125BB014F296A
:10028000491C44294F254F29C91C48296D254F2950
:10029000491D4C2930254F29C91D4F293725C90132
:1002A0007C28BB1B7D290508F039BA008919BE13CB
:1002B000891DBE173A1A75290730BB07BA1A752966
:1002C0000730BB073A1B6E291F303B05143C03194E
:1002D0006C290D30BB027D29BB0A7D291F303B05EF
:1002E000143C031D7529BE1F6C293B1B7D29BB17C0
:1002F000063081001930A0008B1608003B081F391A
:10030000BC003D18862938188A293814BF23B60145
:10031000C001BD010A303C020318C429CA18C32910
:100320004A1C9529CA1EC3299E29B61F9E29BF2390
:10033000B613381D9E29380E0339B2000430C100AF
:100340000310B10DB00DC10BA0293C08B104CA1AAD
:10035000C3293008F0390319B129A03C031DC32972
:10036000B329A030B00430080F390319BB290A3C67
:10037000031DC329BD290A30B0043108F039031D1B
:10038000C329A030B1047F2B0C303C020318D429C0
:10039000B61BBF23B2013C1CB2143C1832140F3000
:1003A000B805320EB8047F2B0E303C020318972A92
:1003B00003304A05031D3E2A4008031D152A310853
:1003C0000F39C2000A3C03191C2A3C18FB290830CB
:1003D0004202031CF229BE1F2B2A09304202031DD0
:1003E0002B2A2C2A42089823E330B605C20D420D71
:1003F0001C39B604122AB30105304202031C0A2A32
:10040000BE1F2B2A09304202031D2B2ABE160F30B5
:10041000B400112A4208A823E030B6054208033987
:10042000B604B814C017C2232B2AC01E1A2A803063
:10043000C0051F2A401B1F2A4B2440172B2ABF230D
:100440003C1C93233C1C2A2ABE1E292A0F30B400D0
:100450002A2AA62340137F2B3108A93C031D332AE7
:10046000BF23CA14962A3108993C031D962A3008E6
:10047000993C031D962ABF234A14962ACA1A542A65
:10048000CA19482A2608B0002708B1004A124D2A86
:100490002808B0002908B1004A164A18522A083024
:1004A000CA06962ACA16962ACA19602A3008310442
:1004B0000319912A3008AD003108AE004916932A7D
:1004C00030080319912A133030020318912A310899
:1004D0000319912A8B132D08C2002608AD0042088B
:1004E000A6002E08C2002708AE004208A700280870
:1004F000AF003008A80070268B1731020319822A3A
:1005000003188B2A8B133108A90091265008A500E7
:100510008B17C916932A2D08A6002E08A7002F08AE
:10052000A8004917962A0830CA06CA127F2B113034
:100530003C020318012BB81C782BBE1EA22A3C18C3
:10054000CB2A782B3C1AAD2A3C1CB2163C18321729
:100550009F30B6053C1CB616B02AB2176030B60400
:10056000320803390319BC2A3308031DF12A381D48
:10057000782BA6239323F12A3308031D782B310807
:100580000F390A3C0319C62AA623E42A34080319A2
:10059000782B3C1AD32A34083C1C8504FF3A3C18BB
:1005A00085053810002B0130B000B1011724B612B8
:1005B000B01784240318762BB013E9239323B213C6
:1005C000321734088504002B3914C6230318782BFE
:1005D0001724B01784240318762BB013E923932330
:1005E000002B3910C6230318782B0319C62A3008AC
:1005F000C200042484240318762B4208B000381566
:100600007F2B031D082BB8103811B601BF237F2B99
:1006100013303C020318472BBE1E102BBE12452B75
:100620000330B408031D182B1C30B30803192A2B00
:10063000C200A03084001430C100801F252B360872
:100640004205000642050319800103308407C10BEF
:100650001D2B3E2BBE1F342BBE0A3E080739053C1E
:10066000031D462BF830BE05A03084003C30C1008D
:100670008001840AC10B382BBE1F8501BE1F452B8C
:100680003E170530BE04BF01462BB8017F2B031D6A
:10069000722BB61B6E2BBE1F512B33080319542B24
:1006A0006E2B330803196E2B3208033903196E2B96
:1006B000B901C6230318782B03196E2BBE1B662BBA
:1006C000B60C360C073903190130A4000424300895
:1006D000AA003108AB00AC01BE1BC916B301B801BA
:1006E000CA017F2B0830BE0638107F2B8830792B4B
:1006F0009930B100B000B201B301B4013D140C3027
:100700003C0203198C2B0D303C0203198C2BC001C9
:10071000BE1E8C2BBE12B40112303C02F830031DF9
:10072000BE053B1708003608C100C10C410C073953
:100730000319A32BC1000130B300C1030319A52B7A
:100740000310B30D9D2B7F30B3000800360803392A
:1007500003190430C1000130B400C1030319B32BE5
:100760000310B40DAD2B08000330B2054030B61EA7
:10077000BD2B2030361FBD2B8030B2040800B201E3
:10078000B301B401AA30B100B00008003008F0395C
:10079000A03C031DD52B0F30B00530080A3C031DCB
:1007A000D52B123039180030B00013303918123000
:1007B00030020318E82B3108F039A03C031DE62B6A
:1007C0000F30B10531080A3C0319E82B60303102C3
:1007D00008003008031DEF2B1230B000F32B12304D
:1007E00030020318F52BB214032C0319022CB000AD
:1007F0000E303002031C022C103030020318022C81
:100800000630B002321408003008123C0319B0015F
:10081000321C162C1230B0071A303002031C162C72
:10082000223030020318162C0630B0070800E330DF
:10083000B6052408BE1B2508C200C20D420D1C3996
:10084000B6042B08B10731080F39093C0630031CE8
:10085000B1073108593C0318302C6030B102B00A9E
:100860002A08B00730080F39093C0630031CB007CE
:100870003008233C03184A2C2430B00236081C39B7
:10088000043E1C390319472C0430B6074A2CE330C8
:10089000B6053615080040081F39C3000030BE1ADF
:1008A00080303C04C200A03084001430C100801F9E
:1008B0006B2CC21B672C36084218622C1C390006B0
:1008C0001C39652C033900060339031D6B2C4308C2
:1008D0000319722CC30303308407C10B572CC016B5
:1008E000BF23832C0008B600840A00087F39B000BB
:1008F000840A0008B100C00AB201BE1BBE1DE92374
:100900009323A623B4230800A03084001430C10030
:10091000801F902C03308407C10B882C03149A2C61
:10092000B61736088000840A30088000840A31082F
:100930008000031008002408BE1B2508D000031007
:10094000D00DD00DA03084001430C100801F162DB2
:1009500000081C390319AF2C5006031D162D000882
:10096000B600840A00087F392A02031D172D840A65
:1009700000082B02031D182D36080339C300031984
:1009800043150130B500C3030319C92C0310B50D7D
:10099000C32C3508B61A8504FF3AB61E8505BE1F5E
:1009A000D52CB61A4914B61EC9148403801FDF2C37
:1009B000361FDC2CB61AE12C84038001162D361F5D
:1009C000172D840320308006840AB61AF92C2625B8
:1009D000F9300002031D172D233080001C30B605AE
:1009E0000319172D0430B602031D112D1C30B6005B
:1009F000112D0008C20080131D25243000020318A9
:100A00008001C21B80177F300005031D172D1C308D
:100A1000B6050319172D0430B607B61E112D043084
:100A2000B6008403E330800536088004840A840A13
:100A3000840AC10BA62C37100800800A00080F3961
:100A40000A3C031D080006308007080000080F3923
:100A500003192C2D80030800800306308002080053
:100A6000F730C7001F30C8006430712508003A25F0
:100A70003A253A25FB30C7009030C800FA3071257E
:100A80000800F630C7000930C8006430712508003E
:100A9000F830C7008930C80064307125080051253E
:100AA0008725F630C7000930C800643071258725D6
:100AB000F830C7008930C800643071250800E23082
:100AC000C7002430C800643071250800E230C70038
:100AD0002430C800FA30712508005F258925662575
:100AE000080083160C1483128C2583160C108312B5
:100AF00008002730C4007C2DC40B7B2D0800033078
:100B0000822D0A30C5007925C50B832D08001E30C3
:100B10008C2D64308C2DFA30C500DD30C400902D52
:100B2000912D922DC40B8F2D0000962D972DC50B66
:100B30008D2D0800FC00030E8301FD000408FF005A
:100B40000A08FE008B18A92D0B19D12D0C18DD2DCC
:100B5000E42D8B10A3030319B92DA21BE42D033040
:100B60004A050319E42D0310210C2302031DE42D73
:100B7000CD2D2108A300A21FC32D0310A30CA30C8D
:100B80000130A206E42DED2DBE1FE42D03304A05F1
:100B9000031DCD2D1030BE06E42D3E120430CA06D2
:100BA000E42D0B1106308100A00BE42D8B12BB1F2E
:100BB000DB2DBB13E42D3B13E42D0C1047088F00F5
:100BC00048088E00803085067E088A007F088400F1
:100BD0007D0E8300FC0E7C0E09002C3084001D2548
:100BE00060302C020318262EBE1F6F2E2B08031D0B
:100BF0001D2E10302C020319162E13302C0203194F
:100C0000192E16302C020319172E19302C02031935
:100C1000192E22302C020319172E25302C0203190D
:100C2000192E28302C0203191B2E1D2ECA144A120D
:100C30001D2E4A161D2ECA104A1259302B02031DB2
:100C40006F2E57302C02031849156F2EAC01371444
:100C50002B3084001D2560302B02031C6F2EAB014E
:100C6000BE1BC9152A3084001D2524302A02031C0E
:100C70006F2EAA01702629020319422E2930840002
:100C80001D255F2E0130A900283084001D2513305A
:100C90002802031D5F2E0130A800273084001D2587
:100CA000A0302702031D5F2EA701263084001D25DA
:100CB000A0302602031D5F2EA6010130A700A40A62
:100CC00008302402031C662E0130A400912650082F
:100CD000A50038186F2E2408BE1B25089823C42DA4
:100CE00002302802031D7D2E2708CD002608CC00E7
:100CF0000F2728304B182930902E04302802031972
:100D00008F2E0630280203198F2E0930280203196E
:100D10008F2E1130280203198F2E3130902E303053
:100D200008000130CD00CC010130D0002608352765
:100D3000D10004305102031CA52E031DA22E27084A
:100D40000319A52E0430D102992E27084D02031D48
:100D5000AD2E51084C020319C22E0130D0070F27C7
:100D60004B18D00A073050020318D0004D308400D1
:100D70001D25A0304D02031DA52ECD014C30840051
:100D80001D25A52E0130CE0028084E020319DC2EA9
:100D90004E083527C200E826D00702304E02031D58
:100DA000D42E0F274B18D00A073050020318D0005A
:100DB0004E3084001D25C42E29083527D007D003C6
:100DC00007305002031CE62ED000E02ED00A0800A7
:100DD000C2030319092FC20303190B2FC2030319FE
:100DE000092FC20303190D2FC2030319092FC203D0
:100DF00003190D2FC2030319092FC2030319092F69
:100E0000C20303190D2FC2030319092FC2030319CB
:100E10000D2F03300E2F00300E2F02300800CB01B3
:100E20004D08C200420E0F39C3000310C30DC30D9D
:100E3000C307C30D42080F3943070339031D342F7D
:100E40004D08031D332F4C08C200420E0F39C3005A
:100E50000310C30DC30DC307C30D42080F39430769
:100E60000339031D342F4B140800C200420E0F3902
:100E7000C3000310C30DC30DC307C30D42080F39D0
:040E8000430708001C
:02400E00C423C9
:02401000FF3F70
:1042000043006F0070007900720069006700680069
:1042100074002000280043002900200032003000F4
:10422000310039002D003200300032003100200012
:104230006200790020004D002E00590061006D00E1
:0A42400061006D006F0074006F0054
:00000001FF
